:020000020000FC
:10000000A5C109C009C009C009C009C00AC018C0FB
:1000100096C196C196C1189518951895189531E016
:1000200018950F930FB70F9308B348E004230023EC
:1000300011F0C39801C0C39A0F910FBF0F9118958B
:100040000F93EF93FF930CB100936000E091610078
:10005000F091620009940BE275D100E373D172D183
:100060000FED70D100E36ED16DD120FF03D003E21C
:1000700069D108950AE366D100E364D163D108959C
:1000800000E360D15FD15ED10FED5CD100E35AD1C6
:1000900059D103E257D108950FE354D153D152D12E
:1000A00003E250D1089500E34DD14CD10AE34AD187
:1000B00000E348D147D1213039F00EE243D100E3CB
:1000C00041D103E23FD108950AE33CD100E33AD1A4
:1000D00039D103E237D108952F9321E0E4DF2F9146
:1000E000089500E32FD12ED10EE22CD100E32AD1C6
:1000F00003E228D108950BE225D100E323D122D1D8
:100100000FED20D100E31ED11DD103E2089500E3DD
:1001100019D118D117D10FED15D100E313D112D198
:1001200020FF03D003E20ED108950AE30BD100E3D0
:1001300009D108D10895063009F4B8C00A3331F462
:100140000AEA0093610000E000936200FF91EF91E2
:100150000F911895073479F00335A1F0063421F09A
:100160000535B9F0A6D0F2CF0CEE0093610000E0A7
:1001700000936200EBCF0FE10093610001E0009378
:100180006200E4CF02E50093610001E000936200A9
:10019000DDCF203019F020E08CD0D8CF21E089D0FD
:1001A000D5CF053611F4C09A15C00E3611F4C19A98
:1001B00011C0033711F4C29A0DC0073711F4C39A66
:1001C00009C0013419F400E3BDD004C0033511F4B3
:1001D00000E3B8D06ED0BACF0B3221F48AD0C59AE2
:1001E0007AD013C00D3221F484D0C59874D00DC0DC
:1001F000013511F47ED009C0033519F47AD051E0ED
:1002000004C0063411F475D052E053D09FCF0536A8
:1002100011F4C09812C00E3611F4C1980EC0033705
:1002200011F4C2980AC0073711F4C39806C003320C
:1002300021F4C098C198C298C3983BD087CF0235AB
:1002400011F431DF2DC0043411F405DF29C00D3461
:1002500031F00E3421F00F3411F0003511F41CDFB1
:100260001FC0043511F43DDF1BC0013411F4F3DE6F
:1002700017C0043611F4EFDE13C0023711F413DF98
:100280000FC00A3511F443DF0BC0043711F433DF1C
:1002900007C0073611F4F4DE03C0033509F41CDF90
:1002A00008D054CF01E34ED004D050CF00E54AD05F
:1002B0004DCF0F9324D030E00BE90093610000E0B4
:1002C000009362000F9108950F9300EC0BBF0F9104
:1002D00008956BBE0895C4980F93513011F403E054
:1002E00001C002E003BF02E008BF02E009BF0F91B6
:1002F00008950F9303B7087F03BF0F9108950F93DD
:100300000EB5087F0EBD0F9108950F931F931EB574
:10031000187F0770102B1EBD1F910F91C79A08956B
:100320000F9309B7006809BF0F9108950F9309B79C
:100330000F7709BF0F9108956CBC6DBC0895189597
:10034000189518955D9BFECF0CB90895F8940FEDA4
:100350000DBF00E0602E262DACDF68BA6CB80FEF41
:1003600007BB00E808BB62BA02EF01BB62BA09E151
:1003700009B9579A549A539AC798C69AC49A52E0A0
:0A038000BEDFD4DFA6DF7894FFCFC4
:00000001FF
